:020000040000FA
:04000000D3303A2897
:08000800A000030EA100831209
:100010008B1C32288B1031181428B11C3228643004
:10002000010203183128182800001628172818285C
:1000300019281A281B281C281D281E281F283110A3
:10004000B114A810031005190314AA0DA90DA80DC9
:10005000B00B322831152A08AF002908AE00280855
:10006000AD00B11081010B11210E8300A00E200EF6
:02007000090085
:0C007400203084008001840A80300402E7
:10008000031C3C281230B0009121850187018316A2
:100090000C308505870183128316051483128501B0
:1000A00087010730990000309A00103083168E00C7
:1000B0008312603083168F00831200308316910004
:1000C0009F008312C8308316810083123130900064
:1000D000003083168C00831210308B0083160030A2
:1000E0009B001C141A088312BC00851D0027831670
:1000F00010309B001C141A088312BD00D721810107
:100100008E018F010B118B100B108C018B17962019
:100110003119AC20B30B9428031085190314B90DC1
:10012000F030390203191E21C023872864003118DA
:1001300008000B1D08000B11B11031141230B00073
:10014000051DA728321483160113831208003210EC
:10015000831601178312080031110130B7008B1389
:100160002030370783169B001C141A088312A40042
:10017000A500C030A5061030370783169B001C145D
:100180001A088312A3000030370783169B001C1443
:100190001A088312A2008B17321CD42822090339B3
:1001A000A200A309A409A50922082D02031D1829EC
:1001B00023082E02031D182924082F02031D1829C5
:1001C00001303702031DE7283D143E14B7210230E9
:1001D0003702031DEE28BD143E14BB210330370245
:1001E000031DF5283D153E14BF2104303702031DC1
:1001F000FC28BD153E14C32105303702031D032919
:100200003D163E14C72106303702031D0A29BD16CC
:100210003E14CB2107303702031D11293D173E1430
:10022000CF2108303702031D1829BD173E14D321F2
:10023000B70A0930370203180800AF283C1C080031
:100240000130B600B300B400B500B70085018701E6
:10025000B1139620B30B4229031085190314B90D6D
:10026000F030390203196929B41F8512B40B4229F1
:100270003708B6080319B600031940298516B603D6
:100280009630B400311D29293111321C4C292D0919
:100290000339AD00AE09AF092F1CB1132F1C29295A
:1002A000B11B29292E182929B1178B1320303707A4
:1002B000BB002F08BA007C2110303707BB002E0886
:1002C000BA007C2100303707BB002D08BA007C2122
:1002D0008B1785018701B70AB60109303702031C65
:1002E0002929D72108003E1C08003E101030BB0011
:1002F0003D08BA007C2108008B133A0883161C15B0
:100300009A0083123B0883169B0055309D00AA304B
:100310009D009C1464009C188A291C1183128B1761
:10032000080000309500603084008B1383160408A9
:100330009B001C141A0883128B178000840A6830F3
:100340000402031C95296430D500E724DC006430E6
:10035000D500EC24DD006430D500F124DE006430EB
:10036000D500F624DF003C30F200F3000800013035
:10037000E800042208000230E800042208000430EB
:10038000E800042208000830E800042208001030C9
:10039000E800042208002030E80004220800403071
:1003A000E800042208008030E80004220800F0176A
:1003B0008B13831670309B001C141A0883128B1742
:1003C000E80004228B13831671309B001C141A085A
:1003D00083128B17E80004228B13831672309B0064
:1003E0001C141A0883128B17E80004228B1383163F
:1003F00073309B001C141A0883128B17E800042228
:100400000430F100F0130800E80803190800681C24
:10041000112A6730D500E724D1006830D500E724E1
:10042000D200E81C1B2A6730D500EC24D1006830CC
:10043000D500EC24D200681D252A6730D500F124B0
:10044000D1006830D500F124D200E81D2F2A673092
:10045000D500F624D1006830D500F624D200681EFD
:10046000392A6A30D500E724D1006B30D500E72463
:10047000D200E81E432A6A30D500EC24D1006B304C
:10048000D500EC24D200681F4D2A6A30D500F12433
:10049000D1006B30D500F124D200E81F572A6A3012
:1004A000D500F624D1006B30D500F624D200F0162A
:1004B000D11A882A511B882A511C672ADC1FF01286
:1004C0005C1F882A501C882AC01B882A0800D11C5F
:1004D000722ADD1FF0125D1F882AD01C882AC11BDA
:1004E000882A0800511D7D2ADE1FF0125E1F882A0F
:1004F000501D882AC21B882A0800D11D882ADF1FA8
:10050000F0125F1F882AD01D882AC31B882A080082
:10051000F01E9E2AF01B9E2A51187030D11871309F
:1005200051197230D11973308B1383169B001C1430
:100530001A0883128B17680203190800D11ABB2A04
:10054000511BBB2A7010511CA92A5014541F70143F
:100550005417D11CAF2AD014D41F7014D417511DB6
:10056000B52A5015D41E7014D416D11DBB2AD0152F
:10057000541E70145416511CC32A511A5016D11A05
:10058000C017511B5012D11CCB2A511AD016D11AA8
:10059000C117511BD012511DD32A511A5017D11A0D
:1005A000C217511B5013D11DDB2A511AD017D11A73
:1005B000C317511BD013F01FE22AD11A0800511B98
:1005C0000800E62AD11A432B511B432B6530D50076
:1005D000521AE724D21AEC24521BF124D21BF6241F
:1005E0005118C400D118C5005119C600D119C7004F
:1005F0006630D500521AE724D21AEC24521BF1249B
:10060000D21BF6245118CC00D118CD005119CE00C0
:10061000D119CF0052085118D700D118D80051195C
:10062000D900D119DA00043070183230F01B3230A2
:100630005118C800D118C9005119CA00D119CB00EE
:1006400051185C14D1185D1451195E14D1195F143E
:10065000F01F3B2B511C2E2B4403C000D11C322B0E
:100660004503C100511D362B4603C200D11D3A2B54
:100670004703C30008005118C001D118C101511926
:10068000C201D119C30151187030D11871305119FC
:100690007230D1197330BB006808E900BA007C21C0
:1006A000BD0108007013851A70178512541885163D
:1006B000071407108512D418851607140710851221
:1006C00054198516071407108512D41985160714B6
:1006D00007108512541A8516071407108512D41AAC
:1006E0008516071407108512541B8516071407106A
:1006F0008512D41B851607140710051605128514DC
:100700008512701B85160800FD010730FF007B086D
:10071000FE0C03188F2BFF0B882BFB0100340310FA
:10072000942BFE0C0318FB07FB0CFD0CFF0B912B0D
:10073000FB0CFD0C003494019301083095008B13E1
:100740008E018F018B17D6135608FB007508F51B19
:10075000FF3CFE00FE138423FD0D7B0DF51FD60725
:10076000F51BD602560876079300031814140930B7
:0407700095000800E8
:1007800002300F02031C0800BF27F4080319E52BF1
:100790006E30D5007419F124F419F6243C18D42BCA
:1007A0007418E724F418EC24E8006818B721E81856
:1007B000BB216819BF21E819C321681AC721E81AAB
:1007C000CB21681BCF21E81BD3210711871087118C
:1007D00007120730F10503308A0071088207F42BF5
:1007E0002C2C642C9C2CD42C0715501CE02C40087D
:1007F000D500571AE724D71AEC24571BF124D71B2E
:10080000F624D6005709F038D40557080F39D61BFF
:10081000D4046108F5006008F6005C1C9B23C80B3B
:10082000E02C4C085C180530C8005C1CC00A5C1049
:1008300044084002031CE02CC01B222C501E222C1A
:10084000C001E02C5012DC1854135C1950105C1DD0
:10085000C0035C1DC017E02C8714D01CE02C41089D
:10086000D500581AE724D81AEC24581BF124D81BB9
:10087000F624D6005809F038D40558080F39D61B8D
:10088000D4046308F5006208F6005D1C9B23C90BC5
:10089000E02C4D085D180530C9005D1CC10A5D10D3
:1008A00045084102031CE02CC11B5A2CD01E5A2CB7
:1008B000C101E02CD012DD18D4135D19D0105D1DDC
:1008C000C1035D1DC117E02C8715501DE02C4208A7
:1008D000D500591AE724D91AEC24591BF124D91B45
:1008E000F624D6005909F038D40559080F39D61B1B
:1008F000D4046508F5006408F6005E1C9B23CA0B4F
:10090000E02C4E085E180530CA005E1CC20A5E105C
:1009100046084202031CE02CC21B922C501F922C52
:10092000C201E02C5013DE18D4125E1950115E1D66
:10093000C2035E1DC217E02C0716D01DE02C430831
:10094000D5005A1AE724DA1AEC245A1BF124DA1BD0
:10095000F624D6005A09F038D4055A080F39D61BA8
:10096000D4046708F5006608F6005F1C9B23CB0BD8
:10097000E02C4F085F180530CB005F1CC30A5F10E6
:1009800047084302031CE02CC31BCA2CD01FCA2CEF
:10099000C301E02C5012DF1854125F19D0115F1DF3
:1009A000C3035F1DC317E02C5223851ED92C85126B
:1009B000E02CE9080319E02C85160310E90CE02C63
:1009C000F10A053071020318F1018F0108000530AA
:1009D0008A00D5135508820005308A00D5175508BE
:1009E000820006308A00D5135508820006308A003E
:0609F000D5175508820036
:100A00000034013403340434053406340834093422
:100A10000A340B340D340E340F34113412341334C1
:100A2000143416341734183419341B341C341D3460
:100A30001E342034213422342434253426342734FF
:100A400029342A342B342C342E342F34303432349D
:100A50003334343435343734383439343A343C343C
:100A60003D343E344034C134C234C334C534C6345A
:100A7000C734C834CA34CB34CC34CD34CF34D0347A
:100A8000D134D334D434D534D634D834D934DA3418
:100A9000DB34DD34DE34DF34E134E234E334E434B7
:100AA000E634E734E834E934EB34EC34ED34EE3456
:100AB000F034F134F234F434F534F634F734F934F4
:100AC000FA34FB34FC34FE34C4346434013401346D
:100AD0001134003401342134003400340134003442
:100AE0000034003400340034003400340034003466
:100AF0000034003400340034003400340034003456
:100B0000FF34FE34FC34FB34FA34F934F734F63471
:100B1000F534F434F234F134F034EE34ED34EC34B2
:100B2000EB34E934E834E734E634E434E334E234F3
:100B3000E134DF34DE34DD34DB34DA34D934D83434
:100B4000D634D534D434D334D134D034CF34CD3476
:100B5000CC34CB34CA34C834C734C634C534C334B7
:100B6000C234C1343F343E343D343C343A343934F9
:100B700038343734353434343334323430342F3439
:100B80002E342C342B342A3429342734263425347B
:100B900024342234213420341E341D341C341B34BC
:100BA00019341834173416341434133412341134FD
:100BB0000F340E340D340B340A340934083406343F
:100BC0000534043403340134C4346434013402344D
:100BD000123400340234223400340034103400342F
:100BE0000034003400340034003400340034003465
:100BF0000034003400340034003400340034003455
:100C0000803413341E3426342C34313436343934A1
:100C10003D34403442344534473449344B344C3409
:100C20004E3450345134533454345534563458348B
:100C300059345A345B345C345D345E345F34603430
:100C400060346134623463346434643465346634EB
:100C5000663467346834683469346A346A346B34AF
:100C60006B346C346C346D346D346E346F346F347B
:100C70006F3470347034713471347234723473344C
:100C8000733474347434743475347534763476341F
:100C900076347734773477347834783478347934F8
:100CA00079347A347A347A347B347B347B347B34D1
:100CB0007C347C347C347D347D347D347E347E34AD
:100CC0007E347E347F347F34C4346434013404345D
:100CD0001434003404342434003400340234003436
:100CE0000034003400340034003400340034003464
:100CF0000034003400340034003400340034003454
:100D000080340034003401340234033404340634B3
:100D100008340A340C340E341134143417341A34B1
:100D20001D342134243428342C342F3433343734D4
:100D30003B343F34433447344B344F3452345634CD
:100D40005A345D346134643467346A346D347034D9
:100D500072347434763478347A347B347C347D3431
:100D60007E347E347E347E347E347D347C347B34F9
:100D70007A34783476347434723470346D346A343E
:100D80006734643461345D345A34563452344F34E9
:100D90004B34473443343F343B34373433342F34CB
:100DA0002C342834243421341D341A3417341434A8
:100DB00011340E340C340A34083406340434033449
:100DC0000234013400340034C4346434013408344F
:100DD000183400340834283400340034203400340B
:100DE0000034003400340034003400340034003463
:100DF0000034003400340034003400340034003453
:100E00003C1C080072147314F1011430B6008512F2
:100E10000730F10507308A0071088207162F242F4A
:100E2000272F372F3A2F4A2F4D2F5D2F6108F500BE
:100E30006008F6000715871087110712D4015414B3
:100E400054175223D601602F7F30D600602F7508CB
:100E5000E1007608E0006308F5006208F60007117B
:100E60008714D401D414D4175223D601602F7F30B5
:100E7000D600602F7508E3007608E2006508F500EB
:100E80006408F60087108715D4015415D416522330
:100E9000D601602F7F30D600602F7508E5007608F8
:100EA000E4006708F5006608F60087110716D4010C
:100EB000D41554165223D601602F7F30D600602FF0
:100EC000741A892F7118692F7419F60A7418F603A9
:100ED0006D2F7419F50A7418F50350307418F20068
:100EE0007419F300C8307602C8300318F600503089
:100EF00076025030031CF600F51F842FA0307502D7
:100F0000A030031CF500892F64307502643003188B
:100F1000F5007F30D600711CD6019B23F001BF275E
:100F2000741C942F731B7416741D982F721B7416E7
:100F3000741E9D2FF10AF119AE2F8512B60BA52F45
:100F400085163C3071180A30B60064000A300F0272
:100F5000031CA52F8F01741A082F602F7508E70056
:100F60007608E600603084000408BB000008BA0080
:100F70007C21840A68300402031CB42F0800F401A9
:100F80000A30851DF2078519F202783072020319C2
:100F9000741479300318F200153072020319F41436
:100FA0001430031CF2000A30051CF3070518F30285
:100FB000783073020319741579300318F300153073
:0E0FC00073020319F4151430031CF30008002B
:084000000B000300040009009D
:02400E00CC33B1
:10420000010003000300030003000200020002009B
:1042100002000000000000000000FF00FF00FF009F
:10422000000000000000000000000000000000008E
:104230000000C000C000C000C000FF00FF00FF0081
:104240000100C300F300CF00FF00C300F300CF0064
:10425000FF00C300F300CF00FF00FF00FF00FF00DE
:10426000FF00FF00FF00FF00FF00FF00FF00FF0056
:10427000FF00FF00FF00FF00FF00FF00FF00FF0046
:10428000FF00FF00FF00FF00FF00FF00FF00FF0036
:10429000FF00FF00FF00FF00FF00FF00FF00FF0026
:1042A000FF00FF00FF00FF00FF00FF00FF00FF0016
:1042B000FF00FF00FF00FF00FF00FF00FF00FF0006
:1042C0007D00FC007D00FC007D00FC007D00FC000A
:1042D000FF00FF00FF00FF00FF00FF00FF00FF00E6
:1042E0000000000000000000FF00FF00FF00FF00D2
:1042F000FF00FF00FF00FF00FF00FF00FF00AA001B
:00000001FF
